:040000008A01032846
:1000060083177D3084007E308A110D208A1183018A
:100016008A11152864008001840A04060319003435
:1000260004060E280030A2000030A3000030A00015
:100036000030A10098130310831603130030031831
:1000460001308500031000300318013086008A1144
:1000560092268A118A11F3278A1183120313200824
:10006600013EA00021080318013E003EA100003019
:10007600A2000030A3003F2820082207013E8A1173
:1000860009278A11B8002208243E83138400380801
:1000960080000130A2070318A30A0030A307230833
:1000A600803AB80080303802031D5B2810302202E7
:1000B600031C5E285F283F28031000300318013018
:1000C600B90000308A1158268A11003083120313B2
:1000D600A2000030A3006F282208243E8313840068
:1000E60000088A11D2258A11831203130130A20750
:1000F6000318A30A0030A3072308803AB80080300B
:100106003802031D882808302202031C8B288C28FD
:100116006F280310003003180130B90001308A112E
:1001260058268A11083083120313A2000030A30058
:100136009C282208243E8313840000088A11D225B5
:100146008A11831203130130A2070318A30A003091
:10015600A3072308803AB80080303802031DB5286B
:1001660010302202031CB828B9289C28C8308A11EE
:10017600D7278A11831203132008103E013E8A11E5
:1001860009278A110038031DC928CA28CE2800303D
:0C019600A0000030A10030288A110328CE
:100BA400B900390886008A11FF258A110D30831295
:100BB4000313BA00DE2DDE2D0130BA02031DE32D2E
:100BC400E42DDD2D0800BE000310003003180130B1
:100BD400BF003E1CEE2DEF2DF32D3D08C000400854
:100BE400BF070310BD0D0310BE0CBE08031DFB2D73
:100BF400FC2DEB2D3F08FE2D0800FD147D0885001B
:100C04001130BB00062E062E0130BB02031D0B2E35
:100C14000C2E052E7D157D0885001130BC00132E89
:100C2400132E0130BC02031D182E192E122EFB3078
:100C3400BE003E08FD057D0885001130BD00232E51
:100C4400232E0130BD02031D282E292E222E08003A
:100C5400FD30C1004108FD057D0885001130BE004E
:100C6400342E342E0130BE02031D392E3A2E332E7B
:100C74007D157D0885001130BF00412E412E0130C5
:100C8400BF02031D462E472E402EFB30C1004108F3
:100C9400FD057D0885001130C000512E512E013014
:100CA400C002031D562E572E502E0800BA000230E3
:100CB40086008A112A268A110A308A11D7278A11B6
:100CC400283083120313BD003A088A11E5258A11DE
:100CD40083120313BC0039083C07BA000310003028
:100CE40003180130B9008B2E143086008A112A268D
:100CF4008A11213083120313BB00812E812E01300F
:100D0400BB02031D862E872E802E0130BC003C08BA
:100D1400B9073A083902031C902E912E762E08004A
:100D240038308312031386008A112A268A1105306B
:100D34008A11D7278A1138308312031386008A1147
:100D44002A268A11213083120313B900AA2EAA2E4F
:100D54000130B902031DAF2EB02EA92E3830860003
:100D64008A112A268A11213083120313BA00BB2E5A
:100D7400BB2E0130BA02031DC02EC12EBA2E38304C
:100D840086008A112A268A11213083120313BB009C
:100D9400CC2ECC2E0130BB02031DD12ED22ECB2E55
:100DA400013086008A112A268A1132308A11D72707
:100DB4008A110D308312031386008A112A268A11A0
:100DC400213083120313BC00E82EE82E0130BC024C
:100DD400031DED2EEE2EE72E063086008A112A26FC
:100DE4008A11213083120313BD00F92EF92E01302C
:100DF400BD02031DFE2EFF2EF82E0800FE00FE1F6E
:100E0400082F83137E188317000808000408FE00C7
:100E140007308A007E08820700342E342E342E34A4
:100E24002E342E342E342E342E34453456344F344E
:100E34004C345534503449344334203442346F34C0
:100E44006F3474346C346F346134643465347234A4
:100E54002034313436344634383438342C34203465
:100E640032343034313431342E342E342E3453343D
:100E740049345334543445344D34413420344D349E
:100E84004934433452344F3443344F344E3454345D
:100E940052344F344C34413444344F3452342E346D
:100EA4002E342E342E342E342E342E342E34453417
:100EB40056344F344C34553450344934433400346C
:100EC400003400340034003400340034003400347E
:100ED400003400340034003400340034003400346E
:100EE400003400340034003400340034003400345E
:100EF400003400340034003400340034003400344E
:100F0400003400340034003400340034003400343D
:100F1400003400340034003400340034003400342D
:100F2400003400340034003400340034003400341D
:100F3400003400340034003400340034003400340D
:100F440000340034003400340034003400340034FD
:100F540000340034003400340034003400340034ED
:100F640000340034003400340034003400340034DD
:100F740000340034003400340034003400340034CD
:100F840000340034003400340034003400340034BD
:100F940000340034003400340034003400340034AD
:100FA4000034003400340034003483120313BE00D0
:100FB4000430BF005330C000E02FE02F0130C002E6
:100FC400031DE52FE62FDF2F0130BF02031DEB2F9A
:100FD400EC2FDC2F0130BE02031DF12FF22FDA2F8C
:100FE400080001308312031386008A112A268A110D
:0A0FF4000A308A11D7278A1108007D
:00000001FF
